:10000000F400FFFFFFFFFFFFFFFFFFFFFFFFFFFF0A
:10002000FFFFFFFFA10EFFFFFFFFD60FFFFFFFFF48
:10003000FFFFFFFFD214FFFFFFFFFFFFFFFFFFFFE8
:100080007E00000000E59DB29927AC37E372A9FF1E
:1000900000080000000A00A00003000000000000AB
:1000A000680000000002050A1000002833394046AD
:1000B0004C52565A5F646A6F74797E83898F949923
:1000C0009DA1A5A8ABAEB1B4B7BA6352431F0063FC
:1000D00052442E1B4D34210B0052372A1E1B4E3E1C
:1000E0003020004E3E302010000000FFFFFFFFFFD9
:1000F000FF00000061D0EE1C1EFE9AE0061000001A
:100100000300FC161FFEA3C0A100BB8BFD169000D0
:100110001494FCC6EAAA00AD0687958684FAF41604
:1001200002FCC6EA94FCAD06A1009786FAF416809C
:100130000014AEFCC6EA8000AD0687958684FAF40A
:1001400016AEFCC6EAAEFCAD06A1009786FAF49A9C
:10015000D301FAFE4D00AD1AB3D289BA61FC253045
:10016000253083B92583B983B82583B88BEE99BA36
:10017000C2B2AF83B85EBC83B883B95EBD83B93009
:100180005EBA305EBB99BAAF1020FE0302FC100CC1
:10019000FC0304FCA1009E06FC9E07FCA10C9E082B
:1001A000FCA1019E09FCA1049E0AFC0A027B1E1010
:1001B00002FC9AF01A9A241B4252BD039A1C1B7A25
:1001C0001E0B02AFB7160000C6EA3C19AD0386FA53
:1001D000F7B6AF9A410FA1059E32FCA1009E74FCB8
:1001E000419E77FC9A450C9A3216311384161B8473
:1001F000AC84059A5003FA0C310384059AEB0CFA8F
:10020000039A1202315384055B849ACF027110FA6B
:10021000D6AF9A65059AFC058C001C149CFC854D94
:1002200000AD14A100958E1AFC9E77FC9AE5169AF3
:10023000AC119AF811FA2531030021149CFC855168
:10024000AD1AA101958E77FC9E1AFCA1009E77FC49
:100250009AE5169AC4119AE9119A69068E83FC4DA3
:1002600000BD141496FC8541954814FC8D06A10030
:10027000959AD90F9A05101498FC8541954899FCD8
:100280008D06A100959A0412149AFC854195489B0D
:10029000FC8D06A100959AC7111497FC85419548DD
:1002A00015FC8D06A100959AB0031494FC85419528
:1002B0004895FC8D06A100959A6F0831230C021B0E
:1002C0000CAC0C07A1014832FC8D039A6906AF31D2
:1002D0001385051B859AAC113163840D9A38084249
:1002E00052BD046B84FA025A843173840D9AA316AA
:1002F0004252BD047B84FA025A84313385139A3505
:10030000054252BD0A3B858E7EFC9E18FCFA025ABD
:10031000843153851F9ADA194252BD169A35054227
:1003200052BD0F8E7EFC9E18FCA1009E7FFC5B855B
:10033000FA025A84310385050B859AE51631238527
:10034000052B859A450C314385054B859ACF12AF15
:10035000AC010B31030358BC01553A84FA519A277A
:10036000149A03079A26199A50198E7DFC9E16FC42
:100370008E7EFC9E18FC9A01054252AD05A1E09EBE
:100380007EFC9A61089A45078E7CFC9E17FC3133EF
:100390008408A1009E7CFC9A38089A36168E74FC5C
:1003A0004D30BD039AC4199A450C9A26162A84AF7B
:1003B0008C03039B5E048C0018CC010E8E1CFC4148
:1003C000AD14141CFC854195FA0CA1009E1CFCFA8E
:1003D00005A1009E1CFCA1009E1EFC9E1DFCBC01F4
:1003E0000E8E1BFC41AD0D141BFC854195FA05A139
:1003F000009E1BFCCC012E3133012A8E1CFC51BD0A
:1004000007A1029E15FCFA538E1CFC4D05BD059AF2
:100410006407FA478E1CFC4D288D409A6407A12082
:100420009E15FCFA363143012DBC012A8E1BFC516E
:10043000BD07A1029E15FCFA228E1BFC4D05BD05D1
:100440009AC507FA168E1BFC4D288D0F9AC507A179
:10045000209E15FCFA05A1029E15FC9B00053103A8
:1004600000039B0005A1009E1CFC9E1BFCCC010E02
:100470008E1EFC41AD0D141EFC854195FA05A100B0
:100480009E1EFCBC010E8E1DFC41AD0D141DFC8595
:100490004195FA05A1009E1DFCCC012E3133012AA5
:1004A0008E1EFC51BD07A1029E15FCFA538E1EFC48
:1004B0004D05BD059A8216FA478E1EFC4D288D40CB
:1004C0009A8216A1209E15FCFA363143012DBC01FB
:1004D0002A8E1DFC51BD07A1029E15FCFA228E1D1D
:1004E000FC4D05BD059A9216FA168E1DFC4D288D01
:1004F0000F9A9216A1209E15FCFA05A1029E15FCEA
:10050000AFB78E7EFC70B1A001B1A0309ADB13B002
:10051000B062764D00BD19A003B150B1A0309ADB96
:1005200013B0B0A014B1A006B1A0309ADB13B0B0E4
:10053000367236B6AFB78E7EFC70B1A001B1A03076
:100540009ADB13B0B08E18FC487EFCAD149A5308A9
:10055000147EFCB5A0029A0A1AB06276367236FA98
:1005600002A200B6AF9C02658E1FFC41AD06141FAF
:10057000FC8541958E9DFC4D00BD268E1FFC488C50
:10058000FC8D1EA1019E9DFC8E77FC310F11147510
:10059000FC856D08950B0C710B2C0A0C710A2CFA5A
:1005A0005A8E9DFC51BD548E1FFC488DFC8D4CA174
:1005B000029E9DFC8E77FC310F411475FC856D0207
:1005C000950B0C710B2C0A0C710A2CFA2E8E9DFCCB
:1005D00051BD208E77FC310F131475FC856D01958C
:1005E0000B0C710B2C0A0C710A2CFA071476FC8583
:1005F0006D0195A1009E1FFC9E9DFCAF8E76FC3187
:100600001F02FA0B8E76FC310F05712B212B01ACEA
:1006100001518E20FC4D029D081420FC854195FA65
:1006200047A1009E76FC1475FC855DF695A1009EA1
:100630007BFC9AC411A1019E77FCA1079E79FC9ACC
:10064000450C9AE516A1009E60FC713BE0714BE001
:100650000A0C710A2C712A212A017A1EA1039E9D7F
:10066000FCFA05A1009E20FCAFB7A6008E16FC4840
:100670007DFCAD29469A53084252AD059AC401FA51
:10068000F4147DFCB5A0009A0A1AB04252AD059A46
:10069000C401FAED9AC4018E7DFC9E16FC8E17FCF7
:1006A000487CFCAD259A3216469A53084252AD0555
:1006B0009AC401FAF49A38084252AD059AC401FA74
:1006C000F49AC4018E7CFC9E17FC664D00AD0F9A17
:1006D00032169A61084252AD059AC401FAF4B6AFD7
:1006E0007B1E13F0049A030F9AF00E9A090F9AE5F5
:1006F000159ACE0E9A2E0F9A7C0F9AA90F9A520F26
:100700007A1EAFA1BA9E72FCA1079E79FCA1109E31
:100710008CFCA1649E8DFCAFB7B1B1891CD6A10041
:10072000BE01AE014D20AD1772B716AA00AAB64998
:1007300002BD05AE0172FA09AE0141BE01FAE3A2A3
:1007400017B0B0B6AFB7B1891CD6C680B1A000B1A2
:10075000A0509A2713B0B0AE01709A1807629E7C21
:10076000FCB0B6AF1475FC856D40958E77FC310FEB
:100770000A0B0C710B2C0A0C710A2C8E7CFC4D1F81
:10078000AD428E77FC317E29A101487CFC8D091495
:100790007CFC850D0295FA1FA104487CFC8D091490
:1007A0007CFC850D0495FA0F147CFC850D0595FAEB
:1007B00006147CFC854195A11F487CFC9D039E7C12
:1007C000FC9A3808AF1475FC856D40958E77FC3126
:1007D0000F0A0B0C710B2C0A0C710A2C8E7CFC4D31
:1007E00000AD548E77FC317E398E7CFC4D0B8D092B
:1007F000147CFC851D0595FA2F8E7CFC4D068D0919
:10080000147CFC851D0495FA1F8E7CFC4D05BD09EA
:10081000147CFC851D0395FA0F147CFC851D049542
:10082000FA06147CFC855195A17F487CFC9D05A1AE
:10083000009E7CFC9A3808AFB78E7CFC5D1F72B7B7
:1008400016AA00AAB676B7A000B1A0509ADB13B0E2
:10085000B0B6AFA000B1A008B1A0509ADB13B0B001
:10086000AFA080B1A008B1A0509ADB13B0B0AFB771
:100870008E32FC9E33FC0242FC0344FC0240FC032B
:1008800042FC023EFC0340FC023CFC033EFC023AFC
:10089000FC033CFC0238FC033AFC0236FC0338FC47
:1008A0000234FC3061013027D20236FC300822FCD1
:1008B000302823FCCA05006143BD033061429D28F6
:1008C0000234FC3061013027D20236FC300822FCB1
:1008D000302823FCDA0500614BBD0330614A9D08D6
:1008E0000234FC0336FCFA130234FC300822FC30DC
:1008F0002823FC21253025300336FC0222FC03345A
:10090000FC0244FC300842FC302843FC300840FC28
:10091000302841FC30083EFC30283FFC30083CFCCD
:1009200030283DFC30083AFC30283BFC300838FCCD
:10093000302839FC300836FC302837FCA2083182D8
:100940000324FC8C000DA1009E46FCA0000348FC83
:100950009B270A1446FC85419551BD039B270A8EAF
:1009600046FC4D02AD039BFD090244FC034AFC0218
:1009700042FC484BFCBD0430484AFC9D060242FC48
:10098000034AFC0240FC484BFCBD0430484AFC9D35
:10099000060240FC034AFC023EFC484BFCBD04300E
:1009A000484AFC9D06023EFC034AFC023CFC484BC4
:1009B000FCBD0430484AFC9D06023CFC034AFC0294
:1009C0003AFC484BFCBD0430484AFC9D06023AFC08
:1009D000034AFC0238FC484BFCBD0430484AFC9DED
:1009E000060238FC034AFC0236FC484BFCBD0430CE
:1009F000484AFC9D320236FC034AFCFA2A8E46FC29
:100A00004D7F9D1D0224FC30184AFC30384BFC03FE
:100A100048FCEA00808D10AD0E1000000348FCFA7F
:100A2000061446FC8551950224FC301848FC3038E9
:100A300049FC4829FCBD04304828FC8D06AD04A6BD
:100A400005FA720224FC301848FC303849FC482B67
:100A5000FCBD0430482AFC8D06AD04A604FA5602FB
:100A600024FC301848FC303849FC482DFCBD0430CB
:100A7000482CFC8D06AD04A603FA3A0224FC30187B
:100A800048FC303849FC482FFCBD0430482EFC8D12
:100A900006AD04A602FA1E0224FC301848FC3038C9
:100AA00049FC4831FCBD04304830FC8D06AD04A63D
:100AB00001FA02A6008E4CFC614EAD0BA1009E4DCA
:100AC000FC669E4CFCFA5C144DFC8541958E9EFCA8
:100AD0004D1E9D18149EFC854195A10A484DFC9D14
:100AE00042A1009E4DFC669E32FCFA37A119484D8A
:100AF000FC9D30A1009E4DFCBC031C8E32FC614E5F
:100B00009D061432FC854195664832FCAD154D00BA
:100B1000BD119E32FCFA0C664832FC9D061432FC74
:100B20008551958E32FC4D00AD2C4D05AD214D0407
:100B3000AD164D03AD0B4D02BD23A1039E78FCFA0B
:100B400021A1079E78FCFA1AA10B9E78FCFA13A14A
:100B50000F9E78FCFA0CA1009E78FCFA05A1019E7C
:100B600078FC9A6D0B9A9F0B9AD80EB6AFA10248EB
:100B700033FC9D114832FC8D0CA010B170B1A082E5
:100B80009ADB13B0B0A1034833FC8D124832FC9DB0
:100B90000DA000B1A002B1A0829ADB13B0B0AF8E5D
:100BA00032FC51BD22149FFC854D00BD1AA1029557
:100BB0001475FC856D20958E77FC310F0A0B0C7136
:100BC0000B2C0A0C710A2C8E77FC311F4D8E32FCD7
:100BD0004D00BD46149FFC854D00BD1CA10395141E
:100BE00075FC856D30958E77FC310F2E0B0C710BDB
:100BF0002C0A0C710A2CFA22149FFC854D02BD1A96
:100C0000A103951475FC856D10958E77FC310F0A44
:100C10000B0C710B2C0A0C710A2C8E32FC4D018DC1
:100C20000E1475FC855DEF95149FFC855DFE958E19
:100C300032FC4D028D0E1475FC855DCF95149FFC22
:100C4000855DFC95AFB7B1B1891CD68E77FC311F9D
:100C50002C8E74FC4D00BD0A10CF00BE0330BE02C6
:100C6000FA458E74FC4D30BD0A10E300BE0330BE61
:100C700002FA3410D900BE0330BE02FA2A8E74FC88
:100C80004D00BD0A10CA00BE0330BE02FA198E74B0
:100C9000FC4D30BD0A10DE00BE0330BE02FA081063
:100CA000D400BE0330BE02A100BE01AE014D05ADB1
:100CB000368E26FCA000300D02D2AE0230AE03D438
:100CC0008561029D0143AE01A0023188CA28FCD48F
:100CD0006295638495AE0230AE0380BE0330BE02DF
:100CE000AE0141BE01FAC4B0B0B6AFB7B1891CD6EF
:100CF0008EA1FC4D03BD039BAA0D4D02AD604D01BD
:100D0000AD384D00AD039BDA0D9A53084252BD2712
:100D10009A22169AA20F9ACF0F9A750F7A015A014A
:100D20006A0113417CA000B1A002B1A0829ADB133A
:100D3000B0B0A1019EA1FC9B9B0E8E74FC4D30BDFA
:100D400007A1029EA1FCFA133103000F7B01A1074A
:100D50009E79FC9AE516A1029EA1FC9B9B0E0222A5
:100D6000FCEA7F028D05AD039B9B0E0222FC5D0019
:100D700030728EA5FC73B7621653FCBBB60222FC20
:100D80005D00D202A2FC30610A30612B03A2FC1488
:100D9000A5FC854D07BD0AA10095A1039EA1FCFA03
:100DA0000614A5FC8541959B9B0E0222FC5D00303C
:100DB000728EA5FC73B762165BFCBBB68EA5FC4DAC
:100DC00003BD0E6B01A1009EA5FCA1049EA1FCFA2F
:100DD0000614A5FC8541959B9B0EAC01039B9B0EC5
:100DE00002A2FCA208318260BE018E74FC4D30BDAF
:100DF00016AE011D19BE01C680B1A0019A0A1AB033
:100E00004252BD0313995AAE0148A4FC9D1A5B01DE
:100E10006A01C680B1A0019A0A1AB04252BD096B9C
:100E2000015A01AE019EA4FC0222FC5D00EA800092
:100E30009D698EA5FC72B71653FCAAB67202A2FC7D
:100E400030611A303D0003A2FC8EA5FC5D0372B731
:100E5000165BFCAAB6728EA5FC73B7621653FCBB78
:100E6000B68EA5FC72B71653FCAAB67202A2FC306D
:100E7000610A302D0003A2FC0222FC5D0030728E5C
:100E8000A5FC5D0373B762165BFCBBB68EA5FC4D7B
:100E9000079D0341FA02A1009EA5FC9AD80EB0B6A8
:100EA000AFB1B3B589B8B189BAB189BCB189BEB1A6
:100EB0007A1E8908A24031820322FC9AE60EB0997C
:100EC000BEB099BCB099BAB099B8B4B2B08F132F74
:100ED00003132890132903AF710A28000000007142
:100EE0007A28710BE6AF710AE6717B28710B28AF87
:100EF000139F00717AA2710BA013A10013FB007164
:100F00001BA0AFB7F4AC76B6AF13311B132003139D
:100F1000211F13220A13230F132C051100001101A6
:100F200004110200110300110C0113480CAF717B76
:100F300043713AE6713BE2138C0613419B13430065
:100F4000AF713BE6717A43AF717B43713AE6713B17
:100F5000E2AF717B6B715AE5715BE1136A03F421B7
:100F60005D7FF621D8017F11177F136B40AF710AA7
:100F70006B717A6BAF717B6B710B6BAF717B69714E
:100F80004AE5714BE11369281118FF111900F4218A
:100F90005DDFF621D801DFAF111900710A69717A9E
:100FA00069AF717B69710B69AF717B6C713AE571E7
:100FB0003BE1136C18111AFF111B00F4215DBFF601
:100FC00021D801BFAF111B00710A6C717A6CAF712F
:100FD0007B6C710B6CAF1A848F31230C12717B6C9C
:100FE000710B6C6B01717B69710B695B01FA158C7C
:100FF000000AA11E9E14FC9A9B10FA08A1A09E1440
:10100000FC9A3B11AF310300108EA6FC4D019D09E7
:1010100014A6FC8541959B9A10A1009EA6FCF01B8E
:101020004862FCAD11F01B4862FC9D04A101FA026C
:10103000A1FF0E1BF21BC81B00BD0A717B6C710B5C
:101040006C6B01FA17C81BFFBD0A6A01717B6C71DA
:101050000B6CFA086B01710A6C717A6CF0194863B9
:10106000FCAD11F0194863FC9D04A101FA02A1FF37
:101070000E19F219C81900BD0A717B69710B695B01
:1010800001FA17C819FFBD0A5A01717B69710B6912
:10109000FA085B01710A69717A69AFB7A1009E64B1
:1010A000FC8E32FC4D028D4DA104187DFC728E32F7
:1010B000FC73B716E800ABB65242AD0421258AFC9A
:1010C0009E62FCA104187DFC728E32FC73B716EE92
:1010D00000ABB65242AD0421258AFC9E63FC3173FD
:1010E000850C7B858E62FCF21B8E63FCF219A100DD
:1010F0009E65FCFA44A1009E62FCF21B8E65FC4DCD
:1011000000BD1AA104187DFC728EEE005242AD049F
:1011100021258AFCF219F0199E63FCFA0F8E65FCFA
:101120004D02BD08111900A1009E63FC1465FC85E9
:1011300041954D04BD03A10095B6AF8E64FC4D10E2
:10114000AD3F4D0CAD3B4D08AD374D04AD334D00BB
:10115000AD2F4D0EAD0C4D0AAD084D06AD044D0240
:10116000BD3CA1024832FC9D0CA1289E62FCA1005E
:101170009E63FCFA29A1009E62FCA1289E63FCFAF2
:101180001DA1024832FC9D0CA1059E62FCA1009E9F
:1011900063FCFA0AA1009E62FCA1059E63FC146434
:1011A000FC8541954D12BD03A10095AF8E66FC4DA7
:1011B00002AD089AC711A1009E9AFC8E7BFC5D03CC
:1011C0009E66FCAF2B02AF31030002FA1B8E7BFC44
:1011D0005D034D02AD0751BD0D2A02FA0B712402C9
:1011E00001712102FA022B02AF8E7AFC310F087BCB
:1011F000011117059A6E0FAFA1009E60FC713BE0D4
:10120000714BE0AF8E7AFC310E0D9A750F7B01A108
:10121000009E60FC9BCE12310300039BCE12313640
:10122000E0043147E00BA1029E60FC713BE0714B92
:10123000E08E7AFC311F5C8E60FC4D00AD5A8E67EB
:10124000FC4D05AD074D03AD0351BD077B019A75FC
:101250000FFA2B8E7DFC4D048D077A019A750FFADB
:101260001DA104187DFC61617210FF00AD0861FCD6
:10127000253025308AF860F2179A6E0F7B011467CB
:10128000FC8541954D20BD46A100951460FC85511B
:1012900095FA3BA1009E60FCA1009E67FC8E7AFC43
:1012A000310F2B8E7DFC4D048D077A019A750FFA54
:1012B0001DA104187DFC61617210FF00AD0861FC86
:1012C000253025308AF860F2179A6E0F7B01AFB790
:1012D0008E83FC5D03BD1E8E32FC7216E800AA9E52
:1012E00062FC8E32FC7216EE00AA9E63FC111B7F1C
:1012F00011197FFA308E83FC310F0A5A01717B6914
:10130000710B69FA08717B69710B695B018E83FC53
:10131000311F0A6A01717B6C710B6CFA08717B6C6E
:10132000710B6C6B01B6AFB7B1B1891CD6711A21C4
:10133000710A211B01711B210B01710B21AE02707F
:101340009A59144252AD101B01711B21710A21716F
:101350001A21A2E09BD713AE08709A5914711A2172
:10136000710A211B01711B210B01710B21AE026D52
:1013700001709A59144252AD0F1B01711B21710A61
:1013800021711A21A2E1FA4F711A21A100BE01AE0A
:10139000014D08AD27AE0A30AE0BD48561019571C1
:1013A0000A213113010AAE0A30AE0BD4856D0195C6
:1013B0000B01710B21AE0141BE01FAD3711A2171EB
:1013C0000A21710A210B01710B211B01711B217173
:1013D0000A21711A21A200B0B0B6AFB7B1B1891C11
:1013E000D6711A21710A211B01711B210B01710B8E
:1013F00021AE02709A59144252AD0F1B01711B218C
:10140000710A21711A21A2E0FA19AE08709A5914D2
:10141000AE0A709A59141B01711B21710A21711AAD
:1014200021A200B0B0B6AFB7A613664D00AD2871CB
:101430001A21710A21711A2131130110711B211B0C
:1014400001711B21710A21711A21FA0B711B210BE9
:1014500001710B2156FAD3B6AFB7B1B1B1891CD621
:10146000A100BE03AE034D08AD24AE04317F05716B
:101470001A21FA051B01711B21710A21AE046101B9
:10148000BE040B01710B21AE0341BE03FAD6711AE3
:1014900021710A21A100BE01BE028C011CAE0130E7
:1014A000AE0280BE0230BE0130EA10278DECADEAFC
:1014B0000B01710B21A2FEFA14311301090B01710A
:1014C0000B21A2FFFA070B01710B21A200B0B0B0F3
:1014D000B6AFB1B3B589B8B189BAB189BCB189BE6B
:1014E000B1715AA69A32163146AA06716AA69BD5E0
:1014F00015100000036EFC3106E31B3107AA0671CC
:101500006AA69BD515026EFC80036EFC6168BDE780
:10151000716AA69BD515715AA6710BE3F4A5709A52
:101520004818629E6BFC3107E331710BE3715AA6D8
:10153000F4A54D4ABD148E6BFC4D19BD0DA1019E45
:1015400077FC9AE5169A0028FADC716AA6F4A57071
:10155000B18E6BFC709A4117B0FA7A3117AA6A8E75
:101560006BFC709A1118629E6DFC100000036EFCFB
:101570003106E3193107AA05716AA6FA58026EFC12
:1015800080036EFC6168BDE8716AA6FA48710BE3DE
:101590003146AA05716AA6FA3C8E6DFCF6A51000CC
:1015A00000036EFC3106E3193107AA05716AA6FA39
:1015B00024026EFC80036EFC6168BDE8716AA6FAC5
:1015C00014710BE3716AA6FA0C3107AA05716AA6B9
:1015D000FA039B2615B099BEB099BCB099BAB099E0
:1015E000B8B4B2B08F717BA6710AE7710BE3710BCF
:1015F000EBF4265DFEF626D806FEF4265DFDF62603
:10160000D806FD13A80813A90013A74A711AAB71D5
:101610000AAB714BA6713AA6712AA6710BE7717AD3
:10162000A6AF717BA6AFA1009E68FC717AA6716A15
:10163000A6AF1399ACAFB7B1891CD6C680B1A000D4
:10164000B1A0829A2713B0B0AE015D1C26265DFCC6
:1016500072AE015D03616A9E73FCAE015DE02125FF
:101660009E74FC9AE5168E7DFC72B716A8FCAAB68D
:101670009E70FC70B1A003B1A0829ADB13B0B0B031
:10168000B6AF8E7DFC41AD06147DFC8541959AA3D5
:1016900016AF8E7DFC4D00AD06147DFC8551959AEC
:1016A000A316AFB7A104487DFC9D039E7DFC8E7DF3
:1016B000FC72B716A8FCAAB6768E70FC614EAD23FC
:1016C000B7A003B1A0829ADB13B0B04252BD12663C
:1016D0009E70FC7A85A1FA9E96FC9E98FCA200FA68
:1016E00002A2E0B6AFB7A6008E77FC310F06A106C6
:1016F0006166FA04A10261668E74FC4D30AD35312D
:101700000300318E79FC310F04A14061668E79FCB3
:10171000311F04A12061668E79FC312F04A1106174
:101720006631230307712B212B01FA1331130004B7
:10173000A19F6156B7A001B1A0829ADB13B0B0B6E9
:10174000AFB7B1891CD68730AE06D6A11B614E9DBE
:10175000039B0E18664D128D0CC6A100CA72FCD4F4
:1017600067959B0E18664D089D039BEB174D11ADB9
:101770006E4D0EAD5C4D0DAD4E4D0CAD404D0BADF7
:10178000324D0AAD224D09AD144D08BD5C679E7AFD
:10179000FC67314E041B0CFA501A0CFA4C679E7B06
:1017A000FC1A855A84FA67675D1F9E7CFC6A845A1E
:1017B00084FA5B679E7DFC7A845A84FA51679E7E28
:1017C000FC3A855A84FA47679E7FFC5A855A84FA08
:1017D0003D679E80FC675D0151BD330A84FA2F6727
:1017E0009E83FC4A855A84FA25FA23664D05AD147A
:1017F0004D07AD0A4D04BD16679E76FCFA10679E34
:1018000079FCFA0A679E77FC0A852A855A84B0B665
:10181000AFB7D6A100CA72FCD4859E8EFC664DFF80
:10182000AD1B4D06AD0B4D03BD18A1009E75FCFA16
:1018300011BC030E148EFC856D8095FA05A15A9E8D
:101840008EFC8E8EFC72B6AFB7D6665DF09E8FFCB6
:10185000665D0F9E90FCA180488FFC9D05A2FF9BBA
:101860002419A130488FFC8D52A110488FFC8D2483
:101870008E8FFC4D10BD0FA1024890FC8D3B41089E
:1018800090FC729B2419A1024890FC8D2C8E90FC38
:10189000729B24198E8FFC4D20BD0FA1014890FC36
:1018A0008D17A1060890FC72FA7AA1014890FC8D70
:1018B00008A1080890FC72FA6BFA67A160488FFCD7
:1018C0008D3B8E8FFC4D60BD0FA1034890FC8D5267
:1018D000A10E0890FC72FA4C8E8FFC4D50BD0FA1EA
:1018E000014890FC8D3CA10C0890FC72FA36A101D5
:1018F0004890FC8D2DA10A0890FC72FA278E8FFC6F
:101900004D70BD0FA1074890FC8D17A1120890FCE7
:1019100072FA11A1014890FC8D08A11A0890FC727E
:10192000FA02A2FFB6AFB7B1891CD6C680B1A0013A
:10193000B1A0509A2713B0B09A8801AE01317E044D
:101940000A86FA090B861472FC856D0195B0B6AF54
:10195000B7B1B1891CD6A1509E26FCC6CA0300B1FE
:10196000A0019AF41AB04252AD07A1E09E81FCFAA0
:1019700022AE039E92FCAE034D408D06A17049033A
:101980009D07A1E89E81FCFA0AAE039E26FCA101F8
:101990009E81FC8E26FC9E82FCC6CA0300B1A0007C
:1019A0009A7C1AB062BE014D00BD0DA10449038DA1
:1019B00007AE039E7DFCFA05A1039E7DFC9ADA1911
:1019C000B0B0B6AF8E92FC4D00AD0E9E26FCA101CC
:1019D0009E81FC8E26FC9E82FCAFB7B1891CD6C6C8
:1019E00080B1A0029A7C1AB06297A10C49019D10A7
:1019F000AE014D338D06A13F49019D04A100BE01FA
:101A0000AE019E7EFC8772B0B6AFB7B1B1891CD66D
:101A1000AE0251AD04310386497B1E9A22169A48C4
:101A20000F9AE60E0A02AE0830AE09B1AE02709A05
:101A3000081BB062BE014D00AD169AA81A9AB41ADE
:101A4000AE0830AE09B1AE02709A081BB062BE019A
:101A50000B029A26169A410F9AD80E7A1EAE017280
:101A6000FA16AE0830AE09D48570B1AE020D027020
:101A7000B1A0509ADB13B0B0B0B0B6AFB7B1891C0B
:101A8000D63103860EAE0630AE07B187709AF41ACF
:101A9000B0FA12AE0630AE07B1870D0270B1A05099
:101AA0009A2713B0B0B0B6AF310386059A201BFA5F
:101AB00002A200AF310386059A1C1BFA02A200AFF6
:101AC0003103860D7B1E9A22169A480F9AE60E0A5B
:101AD00002AF3103860D0B029A26169A410F9AD84F
:101AE0000E7A1EAF310386059A241BFA02A2FFAFBD
:101AF0009A281BAFB7B1891CD6AE0630AE07D4AE5C
:101B000000309A501CB0B6AFB7B1891CD6AE0630C3
:101B1000AE07D4AE00309AA41CB0B6AF9A8A1DAFFF
:101B20009A9F1FAF9A2D20AFB7B5B19AA7234D004A
:101B3000AD05A2F49B491C9A3A24A1FF9EBCFCA1CE
:101B4000009EBDFC9EC5FC8EBDFC9ACA22D69AD8CA
:101B5000224D00AD5B9A11234DFFAD0F8EBCFC4DA5
:101B6000FFBD088EBDFC9EBCFCFA459ACD219ADDD6
:101B7000214D00AD039B351CA1019EC6FC8EBDFC12
:101B8000728EB3FC308EB4FC610A309AF6214D009F
:101B9000AD1B8EC6FC519EC6FCBDE2A1019EC5FCDC
:101BA0008EBDFC9A7C214D00AD039B3C1C9AD52137
:101BB0009A3A248EBDFC4148B7FC9D059EBDFCFAB7
:101BC000868EBCFC4DFFBD62A1009EBDFC8EBDFC9F
:101BD0009ACA22D69A4A234D00BD41B702B0FCD61C
:101BE000A15597869786978697B69ACD219ADD213B
:101BF0004D00BD41C6D48EB3FCA3039A45224D00CF
:101C0000BD059AD521FA238EBDFC9A7C214D00BDDD
:101C10002B9AD5219A3A24A1019EC5FC8EBDFC4188
:101C200048B7FC9D229EBDFCFAA38EC5FC4D00BDAD
:101C300012A200FA149AD521A2FEFA0D9AD521A279
:101C4000FDFA06A201FA02A2FB9A3A24B0B4B6AF9A
:101C5000B7B5B1891CD69A2D244D00AD04A2F3FA74
:101C60003F9A74204DFFAD363087309A2D21EA001F
:101C700000AD2780D2AE0230AE03D4C2D6A200623D
:101C800048B5FC9D078795868442FAF3665D034D4F
:101C900003BD03948795A200FA06A2F7FA02A2FAFE
:101CA000B0B4B6AFB7B5B1891CD69A2D244D00ADEE
:101CB00005A2F39B861D9A74204DFFBD039B711DE9
:101CC0009EBCFC02B0FC3008B9FC302D00D4A1FF52
:101CD000959495949594958772B702B0FCD66297C7
:101CE000B6AE0230AE03D402B0FCD686A200859711
:101CF0008684426248B5FC8DF502B0FC3008B9FC20
:101D0000302D00DA0100D687A00030978630978EFC
:101D1000BCFC9ACA223008BAFC3028BBFC03C0FCC9
:101D2000A1019EC6FC8EBCFC9AE02003C2FC9ACDA9
:101D3000219ADD214D00BD3D02C2FC48C1FC8D074A
:101D40003048C0FC9D3330D48EB9FC738EB3FC9AFE
:101D500045224D00AD2B4D1EAD098EC6FC51AD1D6B
:101D60009EC6FCC43008B9FC302D008003C2FCFACA
:101D7000C7A2FAFA11A2FEFA0AA2F5FA06A2F6FA28
:101D800002A2009AD521B0B4B6AFB7B5B19A3A2441
:101D90009A2D244D00AD05A2F39B981FA1009EC56E
:101DA000FC9A74204DFFBD039B811F9EBCFC8EBC22
:101DB000FC9EBDFC9ACA2203BEFC8EBDFC4148B706
:101DC000FC8D02A10048BCFCBD039B891F9EBDFC8D
:101DD0009ACA2203C0FCD69AD8224D00ADDC8EB23E
:101DE000FC310F509ACD219ADD214D00AD039B852A
:101DF0001FA1019EC6FC8EBDFC728EB3FC308EB45A
:101E0000FC610A309AF6214D00AD238EC6FC519E2E
:101E1000C6FCBDE28EBDFC9A7C214D00AD039B91BA
:101E20001FA1019EC5FC9AD5219A3A24FA8C9AD515
:101E3000219A3A2402C0FCD69A4A234D00AD039B56
:101E4000BA1D02C0FCCA080003C2FCA1009EC6FC69
:101E50008EB6FC41308EC6FC61488D039B131F304B
:101E60008EBCFC9A2D21EA0000BD039B061FD60202
:101E7000B0FCD4A200879586846248B9FC9D0342D9
:101E8000FAF39ACD219ADD214D00AD039B851FA168
:101E9000019EC7FC02C2FCD43008B9FC302D005DA5
:101EA000FC7094655DFC614884AD2602B0FCD6A14F
:101EB000559786978697869702C0FCCA0400D4A3DC
:101EC000038EB3FC9A45224D00BD719AD5219BBA71
:101ED0001D8EB9FC738EB3FC9A45224D00AD184D92
:101EE0001EAD098EC7FC519EC7FCAD50C43008B969
:101EF000FC302D0080FAA0C43008B9FC302D0080E1
:101F000003C2FC9AD5218EC6FC419EC6FC9A3A2497
:101F10009B501E9ACD219ADD214D00AD02FA66023A
:101F2000B0FCD6A1559786978697869702C0FCD4B9
:101F3000A3038EB3FC9A45224D00AD188EBDFC9ACA
:101F40007C214D00BD4B9A3A24A1019EC5FC9AD537
:101F5000219BBA1D02BEFCCA0400D48EB3FCA303AD
:101F60009A45224D00AD0F8EBCFC9A7C214D00BDE0
:101F700020A1019EC5FC8EC5FC4D00BD10A200FA3B
:101F800014A2FAFA13A2FEFA0CA2F8FA0BA201FAB2
:101F900004A2FDFA009AD5219A3A24B0B4B6AFB79C
:101FA000B5B19A2D244D00AD04A2F3FA7C9A7420A9
:101FB0004DFFAD649EBCFC73634D00BD048EB7FC49
:101FC00073538EBCFC614BAD57639ACA22D69AD824
:101FD000224D00ADE3639EBDFC9ACD219ADD214DDB
:101FE00000BD39A1019EC6FC8EBDFC728EB3FC30D3
:101FF0008EB4FC610A309AF6214D00AD278EC6FCE6
:10200000519EC6FCBDE28EBDFC9A7C214D00AD0404
:10201000A2FDFA12A2FCFA0EA2FAFA0DA2FEFA062C
:10202000A2F9FA05A2009AD521B0B4B6AFB7B5B1FE
:102030009A2D244D00BD379A74204DFFAD30729A11
:10204000CA22D6629AE020D4C63008BAFC3028BB37
:10205000FC30611C30613DD6A0008EB9FC3080D4CC
:10206000C6A20030611C30613D8D0542FAF5A2FF29
:10207000B0B4B6AFB7A6006648B7FC9D5F9ACA2257
:1020800003C8FC66A700674D089D167202C8FCB71E
:10209000D6AAB6726773B702B0FCD662BBB647FA6F
:1020A000E5B702B0FCD6AE0030AE01EA5555BD280A
:1020B0008686AE0030AE01EA5555BD1C8686AE0060
:1020C00030AE01EAFFFFBD108686AE0030AE01EAF9
:1020D000FFFFBD04B666FA06B646FA9BA1FFB6AF8F
:1020E000B79ACA22D43008BAFC3008BBFCD603C861
:1020F000FCC4CA0800D4C63018B9FC303D0090D6E4
:10210000614D8D24BD0530614C8D1DB58EB9FCA08F
:10211000003090D4C630610C30612DD485B44DFFB1
:10212000BD06C603C8FCFACE02C8FCB6AFB7307312
:10213000309ACA22D43008BAFC3008BBFCD6C4CAD4
:102140000800D4C63018B9FC303D0090D6614D8DE2
:1021500026BD0530614C8D1FB58EB9FCA0003090B6
:10216000D4C630610C30612DD485B44D00BDD48708
:10217000614BBDCFC6FA03100000B6AFB79ACA22B2
:10218000D402B0FCD6A100BE00BE01BE02BE03A7B1
:1021900001A601A3048EB3FC9A8B224D00BD04A7B7
:1021A00000FA0356BDEDC4CA0400D4A601A3048EF0
:1021B000B3FC9A8B224D00BD04A700FA0356BDED77
:1021C000674D00AD04A1FFFA02A100B6AF7B1E9AD5
:1021D000002D7A1EAF7B1E9A0D2D7A1EAFB3B5026D
:1021E000AEFC9A1A2D9A7B2E624D00AD04A1FFFA27
:1021F00002A100B4B2AFB7B3B5D69A3A24C63072D2
:10220000A100A300B37B1E9AB52D7A1E62B24D1BAE
:10221000BD1E9A3A24C63072A100A300B37B1E9A59
:102220002C2D7A1E62B24D00ADD04D1FADCCFA08F8
:102230004D00AD084D1FADC2A1FFFA02A1009A3AB0
:1022400024B4B2B6AFB7B3B59ECCFCC403CAFC632A
:1022500024245D3F4172A3009A3A2402B0FCD6B711
:10226000B310CAFC7B1E9A8A2E7A1E62B2B64D004B
:10227000AD104D1FADD94D1EAD04A1FFFA06A11E34
:10228000FA02A1009A3A24B4B2B6AFB7B3B59ECC65
:10229000FCC403CAFC635124245D3F4172A3009A2D
:1022A0003A2402B0FCD6B7B310CAFC7B1E9A522D5A
:1022B0007A1E62B2B64D00AD084D1FADD8A1FFFA2F
:1022C000C3A1009A3A24B4B2B6AFB7728EB4FC611F
:1022D0000AA000212727B6AFB7AE004D00BD12AE51
:1022E000014D00BD0CAE024D00BD06AE034D00AD6C
:1022F0001CAE044D00BD12AE054D00BD0CAE064D2A
:1023000000BD06AE074D00AD04A1FFFA02A100B664
:10231000AFB7AE004D55BD2EAE014D55BD28AE0236
:102320004D55BD22AE034D55BD1CAE044DFFBD162F
:10233000AE054DFFBD10AE064DFFBD0AAE074DFF09
:10234000BD04A100FA02A1FFB6AFB7AE004DFFBDBC
:102350002EAE014DFFBD28AE024DFFBD22AE034D96
:10236000FFBD1CAE044DFFBD16AE054DFFBD10AE4A
:10237000064DFFBD0AAE074DFFBD04A100FA02A144
:10238000FFB6AFD6AE054D069D1AAE064D399D146B
:10239000AE074D018D0E4DFF9D0AAE084DFE9D040A
:1023A000A100FA02A1FFAFB110BCFCD6DAAEFCA1CD
:1023B00000969750BDFBB0D69A83234DFFAD6DAE0E
:1023C0000030AE0103AEFC8686AE0030AE0103B035
:1023D000FC8686879EB2FC86879EB3FC86879EB469
:1023E000FCA1049EB7FC86879EB5FC86879EB6FC42
:1023F0008EB5FC41A00030A204318240A104318896
:10240000D490309EB9FC100800A200D630610C3088
:10241000612DEA01049D0342FAF1C603BAFC629EF3
:10242000B8FC8EB2FC61FA9EB2FCA100AF8EB2FC89
:10243000317F04A100FA02A1FFAFB18EB2FC311FBF
:1024400004A1ACF699B0AFFFFFFFFFFFFFFFFFFF56
:10280000B79A5C287A019A002D1020FE9A1A2D9A08
:1028100085284252AD0A5A019A0D2D716AA6FAFE18
:102820007B01A1009EA2FE7A019AC42862764D0027
:10283000AD106A019A0D2D716AA6711BA013994AF9
:10284000FAFE7B019A4D296276317F089A0D2D712F
:102850006AA6FAFE7B01FACFFAFEB6AF713AA6710C
:102860007B6C710B6C6B01717B69710B695B017126
:102870007B6B710B6B711AA07B1EFEE4FFFFFEE603
:10288000FFFF7A1EAFB7A6000A029A7B2E4252AD16
:1028900004A281FA2DA700674D0AAD1F377037B12A
:1028A000A0009AB52DB0624D1BBD0D377037B1A099
:1028B000009A2C2DB062616647FADC664D00AD02CD
:1028C000A282B6AFB7B1B1891CD6710BE3715AA61B
:1028D0003106E3063106AA02FAF63107AA04A2017C
:1028E000FA67F4A54D3ABDE29AD62962BE039AD69C
:1028F0002962BE01A0003030B19AD629B030610AF9
:10290000302D0003A0FE9AD62952BD04A202FA3946
:10291000A100BE02AE0249039D149AD629AE0273ED
:10292000B7621690FEBBB6AE0241BE02FAE69AD678
:1029300029AE024D109D1072B7A1FF1690FEBAB6D7
:10294000AE0241BE02FAEAA200B0B0B6AFB702A032
:10295000FEEA00288D04A202FA7A5A011690FEB708
:10296000A004B110A0FE9A522DB0B04252AD04A204
:10297000C1FA616A0102A0FE5DFCA00024245D3F53
:1029800030B1709A8F2DB04252AD435B011690FE6C
:10299000B7A004B110A0FE9A522DB0B04252AD04BF
:1029A000A2C2FA3002A0FE99B8EEBA0000EEBC0056
:1029B000C0100F009A7301A10A9A5401F0B870B1C7
:1029C000A0009A8F2DB04252AD04A2C3FA066B014B
:1029D0005B01A200B6AFB7710BE3715AA63106E3F3
:1029E00002FAFAF4A5774D308D0CA139614F8D06AE
:1029F000671D3076FA20674D418D0CA15A614F8DCD
:102A000006671D3776FA0F674D618D0AA17A614F0F
:102A10008D04671D577666262626265DF076710B97
:102A2000E3715AA63106E302FAFAF4A5774D308D28
:102A30000DA139614F8D07671D306166FA22674D20
:102A4000418D0DA15A614F8D07671D376166FA10E0
:102A5000674D618D0BA17A614F8D05671D576166CA
:102A6000367236B6AFFFFFFFFFFFFFFFFFFFFFFF2E
:102D000013C0A513C40113C4FE13C401AF13C0A59F
:102D100013C40013C4FF13C400AF22B161F8B6A2FC
:102D2000009A0081A109BE13BE1423AFB7D2891C3B
:102D3000D6AE0473629AC72EAD1122B161F8B0BE4F
:102D400003A2039A008123F0E3FA02A10572A30013
:102D5000B6AFB7D4891CD6AE0473AE0630AE07D674
:102D6000C49AE62EAD2222B1B3B761F8B0BE0560B9
:102D7000BE04B0BE0360BE00B0BE0260BE01A204CD
:102D80009A008123F0E3FA02A10572A300B6AFB75F
:102D9000D2891CD6AE0473629AC72EAD1122B161DE
:102DA000F8B0BE03A2069A008123F0E3FA02A1055F
:102DB00072A300B6AFB7D2891CD6AE0473629AC7AD
:102DC0002EAD1122B161F8B0BE03A2089A00812392
:102DD000F0E3FA02A10572A300B6AFB7D2891CD600
:102DE000AE0430AE05E2D6C2D4AE004D05BD1870BB
:102DF000AE0273AE019AC72EAD153022B5B161F89F
:102E0000B030BE0060FA124D03AD084D04AD04A110
:102E100005FA4722B5B161F8B0BE03B0BE0560BE89
:102E200004A2099A0081234D05BD2D634D00AD28F4
:102E3000324D208D234D309D1F62E4D6AE0170AE21
:102E400002E4BE02A0002626262626273027E430EC
:102E5000611C30613D60BE01F0E372A300B6AF605B
:102E6000B12261F8891CCA0200BE0560BE04A20A34
:102E70009A008123B0F0E372A300AF2261F8A20EA2
:102E80009A008123F0E372A300AFB7D4891CD6AEB9
:102E90000473AE0630AE07D6C49AE62EAD2222B138
:102EA000B3B761F8B0BE0560BE04B0BE0360BE003B
:102EB000B0BE0260BE01A2179A008123F0E3FA02BD
:102EC000A10572A300B6AF334D208D174D309D1371
:102ED00033724D069D0B26262626610B323332FABD
:102EE00002A1FF4DFFAFB7D6AE0070AE01EA008081
:102EF0008D25EA00C09D20753072A000AE024D06FF
:102F00009D10262626262627302730610D302D00DD
:102F1000FA0910FFFFFA043072A100B6EAFFFFAF12
:00000001FF
